:1000000000308A00B82C00000B138B138B1B0528C3
:10001000BE2C46308400000803191D280130A100C1
:10002000A001A00B1128A10B10284A30A000A00BA2
:10003000172800000000800B0E2800343330C00069
:100040003230C1002830C2000630C3000C30C4007A
:100050000130C500F0306500003066000612053042
:10006000C6000920BE013E08053C031C5228403052
:100070003E0784000008BF0086110530C600092035
:10008000BF0E3F08850006160530C600092006127F
:10009000BF0E3F08850006160530C600092006126F
:1000A000BE0A3328BF2C4230A000A00B5528000008
:1000B0000034532086115320BF0E3F088500532083
:1000C000061653200612BF0E3F0885005320061661
:1000D000532006120034532086155320C00E4008CA
:1000E00085005320061653200612C00E40088500D6
:1000F000532006165320061200348030BF005920CA
:100100005030C0006B206130C0006B207230C000E6
:100110006B206130C0006B202030C0006B2061304C
:10012000C0006B206A30C0006B207530C0006B20AF
:100130007330C0006B207430C0006B206130C00091
:100140006B207230C0006B202030C0006B2061300B
:10015000C0006B202030C0006B202030C0006B201E
:10016000C030BF0059206830C0006B206F30C00025
:100170006B207230C0006B206130C0006B202030DB
:10018000C0006B206530C0006B202030C0006B20A9
:100190006130C0006B202030C0006B206430C00094
:1001A0006B206130C0006B207430C0006B20613068
:1001B000C0006B202030C0006B202030C0006B20BE
:1001C0002030C0006B200830BE00FA30C600092085
:1001D000BE0BE5288030BF0059205030C0006B2096
:1001E0007230C0006B206530C0006B207330C000DF
:1001F0006B207330C0006B206930C0006B206F3003
:10020000C0006B206E30C0006B206530C0006B20DA
:100210002030C0006B205330C0006B204530C00040
:100220006B205430C0006B202030C0006B20653044
:10023000C0006B202030C0006B20C030BF005920B0
:100240006330C0006B206F30C0006B206E30C00088
:100250006B206630C0006B206930C0006B207230AC
:10026000C0006B206D30C0006B206530C0006B207B
:100270002030C0006B206530C0006B206D30C000A6
:100280006B202030C0006B204D30C0006B204F3001
:10029000C0006B204430C0006B204530C0006B2094
:1002A0000830BE00FA30C6000920BE0B5229C42C0B
:1002B00001302802F93E03189029073E9129533056
:1002C000AC006530AD006730AE0090295430AC0012
:1002D0006530AD007230AE0090295130AC00753001
:1002E000AD006130AE0090295130AC007530AD00EA
:1002F0006930AE0090295330AC006530AD007830E5
:10030000AE0090295330AC006130AD006230AE00D9
:1003100090294430AC006F30AD006D30AE009029B4
:1003200000340A148A100A1182075F2966296D2990
:1003300074297B29822989298030BF0059203030D7
:100340003307BF00C0006B2030303A07BF00C00049
:100350006B202F30C0006B2030303407BF00C0004E
:100360006B2030303B07BF00C0006B202F30C00037
:100370006B203230C0006B203030C0006B2030303A
:100380003507BF00C0006B2030303C07BF00C00005
:100390006B202030C0006B202030C0006B2020304C
:1003A000C0006B202C08C0006B202D08C0006B2003
:1003B0002E08C0006B20C030BF00592030303107FC
:1003C000BF00C0006B2030303807BF00C0006B207A
:1003D0003A30C0006B2030303007BF00C0006B20C7
:1003E00030303707BF00C0006B203A30C0006B20B0
:1003F00030302F07BF00C0006B2030303607BF0001
:10040000C0006B202030C0006B202030C0006B206B
:100410002030C0006B202030C0006B202030C00096
:100420006B202030C0006B202030C0006B202030BB
:10043000C0006B200034A001A1014608031047183A
:10044000A007A00CA10CC718A007A00CA10C47196D
:10045000A007A00CA10CC719A007A00CA10C471A5B
:10046000A007A00CA10CC71AA007A00CA10C471B49
:10047000A007A00CA10CC71BA007A00CA10C003466
:100480000830A100000000000611831606110000CC
:100490008312C00D8610031C502A83168614831203
:1004A0000318552A831686108312831606158312A5
:1004B000061D582AA10B422A0000061183160611B8
:1004C000000086140000000006158312061D662A2F
:1004D000A10100008618211406118316061183124B
:1004E00086108316861083120034B601AF01B7015F
:1004F000B001B801B1010130B900B201BA00B301D5
:10050000BB00B4010730BC00B5013908A800582170
:100510009C21A501831606178312061FAA2A83169B
:1005200086168312861AA92AB80A3808093C0318C5
:100530009B2AB801B10A3108023C031DA52A3808DC
:10054000043C031DA52AB101B8019C21C830C60096
:1005500009208A2A3108C6000A30C7001B22380841
:100560002107A700831606178312061FB22A9C21B3
:10057000831606178312061FD32A83168616831244
:10058000861AD22AB70A3708093C0318C92AB701C4
:10059000B00A3008053C0318CE2AB0019C21C830AF
:1005A000C6000920B82A3008C6000A30C7001B223E
:1005B00037082107A600831606178312061FDB2AB9
:1005C0009C21831606178312061F022B831686169C
:1005D0008312861A012BBA0A3A08093C0318F22A38
:1005E000BA01B30A3308033C031DFD2A3A08023C52
:1005F000031DFD2AB3010130BA009C21C830C6009A
:100600000920E12A3308C6000A30C7001B223A0835
:100610002107A900831606178312061F0A2B9C21A7
:10062000831606178312061F2F2B83168616831236
:10063000861A2E2BBB0A3B08093C0318212BBB0151
:10064000B40A340B2A2B3B08033C031D2A2BB401AC
:100650000130BB009C21C830C6000920102B340893
:10066000C6000A30C7001B223B082107AA008316D8
:1006700006178312061F372B9C2183160617831239
:10068000061F5C2B831686168312861A5B2BBC0A08
:100690003C08093C03184E2BBC01B50A350B572BFF
:1006A0003C08063C031D572BB5010730BC009C21BC
:1006B000C830C60009203D2B3508C6000A30C700E7
:1006C0001B223C082107AB00831606178312061F66
:1006D000642B3908A80058219C2183160617831221
:1006E000061F862B831686168312861A852BB90A57
:1006F0003908073C03187E2B0130B9003908A800DF
:1007000058219C21C830C60009206D2BBE013E082F
:10071000063C031CAC2B25303E07BF0025303E07AE
:1007200084000008C000C1004108C200C3014208A3
:10073000093C0318A02B0A30C2021030C307A32BB8
:100740004208C307A42B972B4308A1003F0884004D
:1007500021088000BE0A872B1430C60009208316AA
:10076000861400000615000083128610831686107A
:1007700000008312061183160611D0308312C000C8
:100780004022C0014022BE013E08063C031CD12B82
:1007900025303E0784000008BF00C0004022BE0A8A
:1007A000C42B1030C00040228316861000000615AE
:1007B0008312061DD92B00000000000000008316E4
:1007C000861400008312C52C0830C0002008C10028
:1007D00083168614000006158312061DED2B86185D
:1007E0000314861C0310A10D00008316061183124A
:1007F0000611C00BE82B83168614000083128610A6
:1008000041080319062C83168610831200008316F4
:1008100006158312061D0A2C000006118316061108
:10082000000083128610831686108312003483160C
:1008300086140000061500008312861083168610A9
:1008400000008312061183160611D0308312C000F7
:100850004022C001402283168614000006150000C5
:1008600083128610831686100000831206118316E9
:100870000611D1308312C00040220130A000E423D1
:1008800021087F39A5000130A000E42321087F3929
:10089000A6000130A000E42321083F39A700013061
:1008A000A000E42321080739A8000130A000E423B8
:1008B00021083F39A9000130A000E42321081F3995
:1008C000AA00A001E4232108AB00831686100000D3
:1008D00006158312061D6A2C0000000000000000AF
:1008E00083168614000083125821BE013E08063C80
:1008F000031CB72C25303E07BF0025303E0784007F
:100900000008C000C1004108C3000F30C305430800
:10091000C40036303D078400430880004108C3000E
:10092000C2014208033C031C992C0310C30CC20AE9
:10093000912C2F303D078400430880004308C600F7
:100940000A30C7001B222108C300C5004408450720
:10095000C300BD0A3D08063C0318AF2CBD01430887
:10096000A1003F08840021088000BE0A762CC62C16
:1009700084011F30830507309F0004281E28BD0115
:10098000C830C60009207D28752A172C9C21C52C4B
:02099000630002
:02400E00183F59
:00000001FF
